:10000E00323032322D30372D3132202D20313233F5
:05001E00343536370007
:101F07007BFF7A00790E7D2D123069EA494B601FFD
:101F17007BFF7A00790E7D2D123069E92402F9E4FE
:101F27003AFA90018FEBF0A3EAF0A3E9F08004E41A
:101F3700FEFF2290018FE0FBA3E0FAA3E0F99000F7
:101F470001120ED6FF3395E0FEC3EF9430EE6480A6
:101F570094804016D3EF9439EE64809480500B90B0
:101F67000001120ED624D0FF802E900001120ED64B
:101F7700FF3395E0FEC3EF9461EE648094804016D2
:101F8700D3EF9466EE64809480500B900001120E9C
:101F9700D624A9FF80027F00EF7D00FC120EBDFF53
:101FA7003395E0FEC3EF9430EE64809480401ED3F7
:101FB700EF9439EE64809480501390018FE0FBA377
:101FC700E0FAA3E0F9120EBD24D0FF803390018F11
:101FD700E0FBA3E0FAA3E0F9120EBDFF3395E0FEA4
:101FE700C3EF9461EE648094804013D3EF9466EE60
:101FF700648094805008120EBD24A9FF80027F00E0
:10200700EFC454F04CFC90018FE0FBA3E0FAA3E08F
:10201700F9900002120ED6FF3395E0FEC3EF94301D
:10202700EE648094804016D3EF9439EE64809480F8
:10203700500B900002120ED624D0FF803990018FEA
:10204700E0FBA3E0FAA3E0F9900002120ED6FF33FB
:1020570095E0FEC3EF9461EE648094804016D3EF61
:102067009466EE64809480500B900002120ED62482
:10207700A9FF80027F00EF75F010A4FFE5F04CFE8A
:10208700EF4DFF90018FE0FBA3E0FAA3E0F990008A
:1020970003120ED6FD3395E0FCC3ED9430EC64805B
:1020A70094804016D3ED9439EC64809480500B9063
:1020B7000003120ED624D0FD803990018FE0FBA3D8
:1020C700E0FAA3E0F9900003120ED6FD3395E0FC89
:1020D700C3ED9461EC648094804016D3ED9466EC74
:1020E70064809480500B900003120ED624A9FD80C3
:0620F700027D00EF4DFF29
:0120FD0022C0
:10172000E47880F61235C7C286E4F5A775E101F5C5
:10173000E275E34043C91090018DF0A3F090018E53
:10174000E004F0700690018DE004F090018DE070EF
:1017500004A3E0640E70E643B28FE4F5A91235836A
:10176000E4FF12356243EF04E490018DF0A3F090A2
:10177000018DE0FEA3E0FFC39401EE940050157DBF
:101780000112349B90018EE004F070E390018DE033
:1017900004F080DBE4F520C20AC208C20EC20DC20A
:1017A0000CD20F7880F608F67826F618F6782CF624
:1017B00090018DF0A3F090018DE0FEA3E0FFC3EE59
:1017C0009401501C74002FF58274003EF583E4F000
:1017D00090018EE004F070DE90018DE004F080D680
:1017E000E490018DF0A3F090018DE0FEA3E0FFC333
:1017F0009440EE9400501C74002FF58274013EF565
:1018000083E4F090018EE004F070DC90018DE00440
:10181000F080D41235FBE4F5A7E5EF54027010E533
:10182000EF5408D39400748094804003D38001C3A4
:1018300092037D08E4FF1234F8E4782BF67823F65F
:10184000900172E0FBA3E0FAA3E0F97823E6FF75CC
:10185000F010A4F58285F083120ED6FE782B26F6C2
:10186000EE600578230680D8D3EF940074809480CE
:101870004035900172E0FBA3E0FAA3E0F990000D7F
:101880001210EE120EBDFF7455120F03120EBD643E
:10189000556002D20C74AA120F03120EBD64AA6026
:1018A00002D20CEF120F03E5EF5402D394007480C0
:1018B000948040047F018002E4FF12224290018C58
:1018C000EFF090018CE05401703CC20974FF782E57
:1018D000F608F608F608F67E007F107D007B007A99
:1018E00000793412125E90019274FFF0A37425F017
:1018F000A374B0F0A3E4F0A37410F07B007A007935
:10190000341231C08002D209121F077832A60608AD
:10191000A60790018CE0540260030219F1A3F0A322
:10192000F090018EE0C4F8540FC868FF90018DE07C
:10193000C454F048FE900172E0FBA3E0FAA3E0F982
:101940008F828E83120ED670030219E8E92FF9EA0E
:101950003EFA900004120ED620E27CE490018BF057
:1019600090018BE0FDC3781A96506C90018EE0C414
:10197000F8540FC868FF90018DE0C454F048FE9001
:101980000172E0FBA3E0FAA3E0F98F828E83120ECE
:10199000D6FF7E00C006C0077C0090018EE0C4F830
:1019A000540FC868FF90018DE0C454F048FEE92F41
:1019B000F9EA3EFA90000D1210EE782BE68DF0A4B5
:1019C00029F9EA35F0FA7D00D007D00612125E90B0
:1019D000018BE004F0808990018EE004F0700690A5
:1019E000018DE004F00219217F011230E3C20B8067
:1019F00007E4FF1230E3D20BE490018DF0A3F090E6
:101A0000018DE0FEA3E0FFC39401EE940050197A2B
:101A1000007B967D03122EDE90018EE004F070DFD5
:0E1A200090018DE004F080D71235F00235EA17
:0535F600782CE6FF2225
:0635EA00EF24FF920F2206
:0635F000A20FE433FF22EC
:030023000220FEBA
:1020FE00C0E0C0F0C083C082C0D075D000C000C0A8
:10210E0001C002C003C004C005C006C00730995606
:10211E00C2997826067926E77881667021F67826A8
:01212E00F6BA
:10212F00900175740AF0900175E0D3940074809457
:09213F0080400600E014F080ED80
:04214800C2868028A3
:10214C009001757414F0900175E0D3940074809430
:09215C0080400600E014F080ED63
:102165007826E62400F582E43401F583E0F599202C
:102175009803022227209A08200A05C298022223E2
:10218500C29A7825E6062400F582E43400F583E555
:1021950099F0C298E6FF7E0064017012900000E09D
:1021A500FD7003F6807CED54072402782DF6EF646C
:1021B500024E700E782DE664097007900001E02448
:1021C50003F67825E6FFFD7C00B40007ECB40103B7
:1021D500F6804FEFC3782D964048ED24FFFDEC3493
:1021E500FFFC7B017A007900122BD77825E624FFC6
:0F21F500F582E434FFF583E06F60047600802309
:102204009001757414F0900175E0D3940074809477
:0922140080400600E014F080EDAA
:10221D00782A0612002678257600D007D006D0053C
:10222D00D004D003D002D001D000D0D0D082D08342
:05223D00D0F0D0E032FA
:0535FB00782AE6FF2222
:102C8700900001E075F010A4FF900172E0FBA3E053
:102C9700FAA3E02FF9EA35F0FA90000D1210EE9042
:102CA7000178782CE6FF18E68FF0A4FFE02FF58275
:0F2CB700E435F0F583120ED6FF7B017A017976B2
:102CC600900185EFF0A3EBF0A3EAF0A3E9F0900101
:102CD60086E0FBA3E0FAA3E0F9EA494B6022900103
:102CE60086A3A3120EBDFF900185E0FD7C00123580
:102CF600B8900186E0FBA3E0FAA3E0F9EF120F0318
:102D06009001897414F0900189E0D3940074809442
:092D160080400600E014F080ED9D
:102D1F00900185E0F5997F011234663099FDC299D3
:012D2F002281
:103228009001007478F07825E624FFF582E434FFF5
:09323800F583E0900101F07F0232
:1032410090FFFF121144EFF090FFFF121144850827
:0B32510083850982A3E07881F6D28615
:10325C008508838509827414F0850883850982E0CA
:0F326C00D3940074809480400600E014F080EA50
:0C327B00900100E0F5999000020211445F
:10333400C9EFC9E964017028EDC39B403F781AE6E0
:10334400FFEB2FFFE433FEEDC39FEE6480F874803F
:10335400985029D20AC3ED9B782CF678277601225F
:10336400CFE9CFEF6402701ACFEBCFCEEDCEEE6F84
:10337400700AD20A782CF67827760222C20AE478F8
:0333840027F62207
:102DC600900185ECF0A3EDF0C9EFC9BAFF19BBFF7E
:102DD60016900185E06A7003A3E06B7068D20A78EA
:102DE6002CF67827E9F622E964017035C39001864E
:102DF600E09B900185E09A4026781AE62BFFE43A9C
:102E0600FEE0FCA3E0FDC39FEC9E5013D20ACFEB7D
:102E1600CFCEEDCEC3EE9F782CF6782776012280B2
:102E260024CFE9CFEF64027022CEEACECFEBCF906B
:102E36000185E06E7003A3E06F700AD20A782CF663
:0C2E46007827760222C20AE47827F622E0
:10002600900000E0FE54F8900177F0EE12111E00E9
:100036007209007F0A009210009B1100AC1200C3E7
:100046001900D91A00FE2001042801A52902F3335C
:10005600033437037439038E4103994903A45003CB
:10006600F86102BD7003F09800000428900001E0DA
:10007600FD782FE6FB7F018027900001E0FCA3E0DE
:10008600FD782EE6FA08E6FB7F01802BD20A782758
:100096007603020428900001E0FD7831E6FB7F023A
:1000A600123334020428900001E0FCA3E0FD78300E
:1000B600E6FA08E6FB7F02122DC60204289000012C
:1000C600E0FD782FE6FB7F01123334200A03020499
:1000D60028801A900001E0FCA3E0FD782EE6FA08DD
:1000E600E6FB7F01122DC6200A03020428900100B8
:1000F6007478F07F0102042575EF10020428C2AC63
:10010600E4900176F0D2867B017A0179767F7F12C0
:100116002CC67B017A0179767F18122CC67B017A70
:100126000179767F05122CC67823E6122CBF782E2D
:10013600E6122CBF782FE6122CBF7830E6122CBFC1
:100146007831E6122CBF7832E6122CBF7833E612ED
:100156002CBFE4900178F0900178E0FFC39410740E
:10016600809480501074342FF8E6122CBF900178DA
:10017600E004F080E2900176E0FF7B007A007900EF
:03018600122CC672
:10018900900184740AF0900184E0D39400748094FF
:0901990080400600E014F080ED46
:1001A2000202A8900001E0FFC378239640030202F6
:1001B200AFEF75F010A4FF900172E0FBA3E0FAA389
:1001C200E02FF9EA35F0FA900181EBF0A3EAF0A30F
:1001D200E9F0C2ACE4900176F0D2867B017A017933
:1001E200767F7F122CC67B017A0179767F0D122CE5
:1001F200C6900181E0FBA3E0FAA3E0F9120EBD1262
:100202002CBF900181E0FBA3E0FAA3E0F99000018A
:10021200122CBC900181E0FBA3E0FAA3E0F990006C
:1002220002122CBC900181E0FBA3E0FAA3E0F9905A
:100232000003122CBC900181E0FBA3E0FAA3E0F9D9
:10024200900004122CBCE4900178F0900178E0FF59
:10025200C39408748094805026900181E0FBA3E04F
:10026200FAA3E02405F9E43AFA7E00E92FF9EE3A1E
:10027200FA120EBD122CBF900178E004F080CC90EF
:0D0282000176E0FF7B007A007900122CC6A7
:10028F00900184740AF0900184E0D39400748094F8
:09029F0080400600E014F080ED3F
:1002A800C286D2AC0204289001007478F0E4A3F06E
:1002B8007F020204251235E0784412108C90010068
:1002C800747CF07844E6A3F008E6A3F008E6A3F00F
:1002D80008E6A3F07C007D057B017A017900122BEA
:1002E800D7900105EFF07F06020425900001E0FF9A
:1002F8007E006401700FA3E0FDA3E0782ECDF60820
:10030800EDF60203F0EF64024E700A900002E07806
:100318002EF60203F0900001E06403700CA3E0FFE6
:10032800A3E07830CFF608EFF60203F0E490017806
:10033800F0900178E0FFC394107480948050279067
:100348000001E0FEEFC39E501D900178E02402F505
:1003580082E43400F583E0FE74342FF8EEF6900161
:1003680078E004F080CBE47843F6807C7A007B3236
:100378007D01782CE6FF122EDE900001E0FDE4FFFF
:100388001234F8020428900001E024FF92020204CB
:1003980028900001E024FF9201020428782CE660EE
:1003A8000890017A7402F0800E90017A200D05748D
:1003B80003F080037401F09001007479F090017AE1
:1003C800E0900101F07C007D027B017A0179001246
:1003D8002BD7900102EFF07F0312324190017AE0AF
:1003E8006401703CD20E8002D208788076F18030A9
:1003F8007A007B327D017F00122EDE900100747935
:10040800F0900001E0900101F07C007D027B017A10
:10041800017900122BD7900102EFF07F03123241CD
:10042800900177E064A060030206D5781AE66401BB
:10043800700D300F0AFA7B327D017F01122EDE909B
:100448000000E064A1600302057FA3E0C37823965F
:100458004003020574900172E0FBA3E0FAA3E0F9FF
:10046800900001E0FF75F010A4F58285F083120E6C
:10047800D690017AF0EF75F010A4FFE92FF9EA356C
:10048800F0FA900004120ED630E23C900001E0FF32
:1004980012000390017AEFF0900100747FF0A3EF4F
:1004A800F02402FDE433FC7B017A017900122BD79A
:1004B80090017AE0FE2402F582E43401F583EFF03E
:1004C800EE2403FF0206D2900001E0FF120003C2EF
:1004D800ACE4900176F0D28690017AE0D394067469
:1004E80080948040377B017A0179767F7F122CC611
:1004F80090017AE0122CBFE4900178F090017AE044
:10050800FF900178E0C39F500B122C87900178E090
:1005180004F080E890017AE004F0802690017AE007
:100528002478122CBFE4900178F090017AE0FF90D3
:100538000178E0C39F500B122C87900178E004F0FB
:1005480080E8900176E0FF7B007A007900122CC6E3
:10055800900184740AF0900184E0D394007480942C
:0905680080400600E014F080ED73
:100571000206C49001007478F07F010206D2900057
:1005810000E064A260030206D57823E6FFA3E0FE43
:10059100C39F40030206CAA3E0FDC39F40030206B6
:1005A100CAEE9D40030206CA900001E0900178F076
:1005B100E490017FF0A3F0900002E0FE900178E06A
:1005C100FFD39E5034120003900172E0FBA3E0FAC6
:1005D100A3E0F9900178E075F010A4F58285F0832D
:1005E100120ED6FF900180E02FF090017FE03400E1
:1005F100F0900178E004F080BEC2ACE4900176F0A6
:10060100D2867B017A0179767F7F122CC690017F99
:10061100E0FEA3E0FFC39480EE94005002800F90AF
:10062100017FE04480122CBF90017FA3E0FF122CD8
:10063100C0900001E0900178F0900002E0FF90018D
:1006410078E0D39F5056E4A3F0900172E0FBA3E061
:10065100FAA3E0F9900178E0FF75F010A4F5828526
:10066100F083120ED6FE900179E0C39E5026EF75FD
:10067100F010A4FF900172A3A3E02FF9EA35F0FA7C
:1006810090000D1210EE900179122CA9900179E0E1
:1006910004F080B5900178E004F0809D900176E04F
:0A06A100FF7B007A007900122CC6DE
:1006AB00900184740AF0900184E0D39400748094D8
:0906BB0080400600E014F080ED1F
:1006C400C286D2AC800B9001007478F07F011232A4
:1006D40041900177E064587057FA7B327D01782CA1
:1006E400E6FF122EDE9001887401F0A37401F0A3DA
:1006F4007401F07B017A0079011233D790017AEF0B
:10070400F0E0FE2478900100F0EE2401FDE433FCD7
:100714007B017A017900122BD790017AE0FE240143
:10072400F582E43401F583EFF0EE2402FF12324146
:10073400900177E0FF64806008EF64886003020939
:1007440042300F367827E66401700EFA7B327D0161
:10075400782CE6FF122EDE8021E4900178F09001DF
:1007640078E0FFC3781A9650117A007B327D01122B
:100774002EDE900178E004F080E4900000E054075D
:1007840090017AF06407701290017904F0900001EE
:10079400E090017AF09000028008E4900179F090F2
:1007A4000001E090017BF090017AE014F0A3E0FFF7
:1007B400C37823964003020942900172E0FBA3E050
:1007C400FAA3E0F975F010EFA4F58285F083120E18
:1007D400D6FF90017AE0D39F4002EFF07827E664D9
:1007E40001700D782CE690017EF090017DF0800B75
:1007F400E490017DF0781AE614A3F090017DE0788E
:100804002CF690017EE0FF782CE6D39F400302098A
:1008140030E4900178F090017AE0FF900178E0C331
:100824009F400302092290017BE075F010A4FF9021
:100834000172E0FBA3E0FAA3E02FF9EA35F0FA90A5
:100844000004120ED630E203020919900001120EC0
:10085400D66438705390017AE0D394047480948001
:10086400900178E0FF4010A3E02F2402F582E434E5
:1008740000F583E0FD807E7825E6C39FFFE49400C5
:10088400FE74FE2FF58274FF3EF583E0FD90017B3C
:10089400E075F010A4FF900172E0FBA3E0FAA3E07E
:1008A4002FF9EA35F0FA804D900172E0FBA3E0FAEB
:1008B400A3E0F990017BE075F010A4F58285F08344
:1008C400120ED6FF7825E6C39FFFE49400FE900144
:1008D40078E07C002FFFEC3EFE74FF2FF58274FF5E
:1008E4003EF583E0FD90017BE075F010A4FFE92F55
:1008F400F9EA35F0FA90000D1210EE782CE6FF18A4
:10090400E68FF0A4FF900178E02FF582E435F0F54E
:1009140083ED120F15900178E004F002081A90019B
:100924007BE0FF122793782C0602080690017DE0F5
:10093400782CF6900177E0648870031232289001D5
:1009440077E064A86003020AE6300F367827E6648D
:1009540001700EFA7B327D01782CE6FF122EDE80C8
:1009640021E4900178F0900178E0FFC3781A965062
:10097400117A007B327D01122EDE900178E004F0C2
:1009840080E4900001E030E718547FFEA3E0FDED21
:10099400FF90017FEEF0A3EFF09001797403F080F3
:1009A40013900001E0FF90017FE4F0A3EFF09001C9
:1009B400797402F0900179E0FF2400F582E43400B8
:1009C400F583E0FE74012FF582E43400F583E090B2
:1009D400017CF0CFEECF90017BEFF090017CE0FF43
:1009E40090017BE0FED39F4003020AE3EEC3782329
:1009F400964003020ADA900172E0FBA3E0FAA3E056
:100A0400F975F010EEA4F58285F083120ED69001EC
:100A14007AF07827E66401700D782CE690017EF078
:100A240090017DF0800BE490017DF0781AE614A328
:100A3400F090017DE0782CF690017EE0FF782CE6C2
:100A4400D39F4003020AC8E4900178F090017AE051
:100A5400FF900178E0C39F505D90017BE075F0103A
:100A6400A4FF900172E0FBA3E0FAA3E02FF9EA35BA
:100A7400F0FA900004120ED620E233900178E0FFE1
:100A8400A3E02F2402F582E43400F583E0FD900016
:100A94000D1210EE782CE6FF18E68FF0A4FF9001FB
:100AA40078E02FF582E435F0F583ED120F1590010F
:100AB40078E004F0809690017BE0FF122793782C75
:100AC40006020A3C90017DE0782CF690017AE0FF62
:100AD400900179E02FF090017BE004F00209DF122D
:020AE4003228B6
:010AE60022ED
:10F000007880E664F1600302F805784EF608F67839
:04F0100081E6602A0B
:10F0140090018B740AF090018BE0D3940074809477
:09F0240080400600E014F080EDCC
:10F02D00784F06E618700106784EB627D508B6104B
:10F03D00D1C2AFE4784AF618F620983CE4784EF643
:10F04D0008F620982FC3784FE6948818E69413504D
:01F05D00238F
:10F05E0090018B740AF090018BE0D394007480942D
:09F06E0080400600E014F080ED82
:10F07700784F06E61870D10680CEB29680C17849DF
:10F08700A699C298E6FF641A6008EF640A60030253
:10F09700F1AFE4784EF608F620982FC3784FE69440
:07F0A7008818E694135023C2
:10F0AE0090018B740AF090018BE0D39400748094DD
:09F0BE0080400600E014F080ED32
:10F0C700784F06E61870D10680CE20980302F046E6
:10F0D700784AA699C298E4784EF608F620982FC386
:0BF0E700784FE6948818E6941350233D
:10F0F20090018B740AF090018BE0D3940074809499
:09F1020080400600E014F080EDED
:10F10B00784F06E61870D10680CE20980302F046A1
:10F11B00784AA699C298E4784EF608F620982FC341
:0BF12B00784FE6948818E694135023F8
:10F1360090018B740AF090018BE0D3940074809454
:09F1460080400600E014F080EDA9
:10F14F00784F06E61870D10680CE20980302F0465D
:10F15F00784AA699C29818E6641A600302F7F6D2A5
:03F16F0086C299BC
:10F1720090018B7414F090018BE0D394007480940E
:09F1820080400600E014F080ED6D
:06F18B007599783099FD32
:10F1910090018B740AF090018BE0D39400748094F9
:09F1A10080400600E014F080ED4E
:10F1AA00C28602F7F67849E6FF7E006450600302E1
:10F1BA00F282784EF608F620982FC3784FE69488A4
:06F1CA0018E69413502327
:10F1D00090018B740AF090018BE0D39400748094BA
:09F1E00080400600E014F080ED0F
:10F1E900784F06E61870D10680CE20980302F046C3
:0AF1F900784AA699C298D286C299FE
:10F2030090018B7414F090018BE0D394007480947C
:09F2130080400600E014F080EDDB
:08F21C007599793099FDC29942
:10F2240090018B7414F090018BE0D394007480945B
:09F2340080400600E014F080EDBA
:08F23D007599013099FDC29999
:10F2450090018B7414F090018BE0D394007480943A
:09F2550080400600E014F080ED99
:06F25E00E4F5993099FD72
:10F2640090018B740AF090018BE0D3940074809425
:09F2740080400600E014F080ED7A
:0FF27D00C28602F7F6EF64014E7062D286C29924
:10F28C0090018B7414F090018BE0D39400748094F3
:09F29C0080400600E014F080ED52
:08F2A5007599783099FDC299BA
:10F2AD0090018B7414F090018BE0D39400748094D2
:09F2BD0080400600E014F080ED31
:06F2C600E4F5993099FD0A
:10F2CC0090018B740AF090018BE0D39400748094BD
:09F2DC0080400600E014F080ED12
:10F2E500C28602F7F67849E66402600302F3E6781F
:10F2F5004EF608F620982FC3784FE6948818E694C2
:03F305001350237F
:10F3080090018B740AF090018BE0D3940074809480
:09F3180080400600E014F080EDD5
:10F32100784F06E61870D10680CE20980302F04689
:10F33100784AA699C298E408F618E6FF13B39296A4
:10F34100EF25E0FECC74F0CCCD7400CDC3E49DEE8E
:10F351009C502AE67F0025E0FEC39460501FE4F52F
:10F36100A7758F037850EEF608EFF675B7A578808C
:10F37100E6F5B78F828E83E4F0F58F8004784B76C3
:05F38100FFD286C299D5
:10F3860090018B7414F090018BE0D39400748094F8
:09F3960080400600E014F080ED57
:08F39F007599783099FDC299BF
:10F3A70090018B7414F090018BE0D39400748094D7
:09F3B70080400600E014F080ED36
:08F3C000784BE6F5993099FD48
:10F3C80090018B740AF090018BE0D39400748094C0
:09F3D80080400600E014F080ED15
:10F3E100C28602F7F67849E66403600302F5757890
:10F3F1004EF608F620982FC3784FE6948818E694C5
:03F4010013502382
:10F4040090018B740AF090018BE0D3940074809483
:09F4140080400600E014F080EDD8
:10F41D00784F06E61870D10680CE20980302F0468C
:10F42D00784AA699C298E4784EF608F620982FC32C
:0BF43D00784FE6948818E694135023E3
:10F4480090018B740AF090018BE0D394007480943F
:09F4580080400600E014F080ED94
:10F46100784F06E61870D10680CE20980302F04648
:10F47100784CA699C298784AE6FF139296EF25E058
:10F48100FECC74F0CCCD7400CDC3E49DEE9C400362
:10F4910002F046E625E0FCC39460400302F046E436
:10F4A100F5A7758F01784CE675F020A42400FFE5DF
:10F4B100F03C7850F608EFF6E4784DF6784DE6C367
:10F4C1009420748094805047E408F608F62098163A
:10F4D100C3784FE6948818E69413500A000806E6AC
:10F4E1001870EA0680E720980302F04675B7A57800
:10F4F10080E6F5B778500806E618CEE6CE7001062C
:10F5010014F5828E83E599F0C298784D0680ADE4BA
:06F51100F58FD286C299BD
:10F5170090018B7414F090018BE0D3940074809465
:09F5270080400600E014F080EDC4
:08F530007599783099FDC2992C
:10F5380090018B7414F090018BE0D3940074809444
:09F5480080400600E014F080EDA3
:06F55100E4F5993099FD7C
:10F5570090018B740AF090018BE0D394007480942F
:09F5670080400600E014F080ED84
:10F57000C28602F7F67849E6FD7C00640460030267
:10F58000F664784EF608F620982FC3784FE69488F4
:06F5900018E6941350235D
:10F5960090018B740AF090018BE0D39400748094F0
:09F5A60080400600E014F080ED45
:10F5AF00784F06E61870D10680CE20980302F046F9
:10F5BF00784AA699C298E625E07852F608E4F678DC
:10F5CF004BF6784EF608F678520806E618CEE6CED9
:10F5DF0070010614F5828E83E493784B26F6784FEC
:10F5EF0006E618700106784FE6700418E66402709C
:05F5FF00D6D286C2997E
:10F6040090018B7414F090018BE0D3940074809477
:09F6140080400600E014F080EDD6
:08F61D007599783099FDC2993E
:10F6250090018B7414F090018BE0D3940074809456
:09F6350080400600E014F080EDB5
:08F63E00784BE6F5993099FDC7
:10F6460090018B740AF090018BE0D394007480943F
:09F6560080400600E014F080ED94
:10F65F00C28602F7F6ED64054C600302F7EC784EB4
:10F66F00F608F620982FC3784FE6948818E694137F
:02F67F00502316
:10F6810090018B740AF090018BE0D3940074809404
:09F6910080400600E014F080ED59
:10F69A00784F06E61870D10680CE20980302F0460D
:10F6AA00784AA699C298E4784EF608F620982FC3AD
:0BF6BA00784FE6948818E69413502364
:10F6C50090018B740AF090018BE0D39400748094C0
:09F6D50080400600E014F080ED15
:10F6DE00784F06E61870D10680CE20980302F046C9
:0AF6EE00784CA699C298D286C29902
:10F6F80090018B7414F090018BE0D3940074809483
:09F7080080400600E014F080EDE1
:08F7110075997F3099FDC29942
:10F7190090018B7414F090018BE0D3940074809461
:09F7290080400600E014F080EDC0
:10F732007599203099FD784AE625E0FC784CE6750B
:10F74200F020A42400FFE5F03C7852F608EFF6E43E
:10F75200784BF6784DF6784DE6C394207480948009
:04F762005048C299B0
:10F7660090018B7414F090018BE0D3940074809414
:09F7760080400600E014F080ED73
:10F77F007852E6FE08E6F5828E83E493F599309988
:10F78F00FD78520806E618CEE6CE70010614F58213
:0FF79F008E83E493784B26F6784D0680ACC299A2
:10F7AE0090018B7414F090018BE0D39400748094CC
:09F7BE0080400600E014F080ED2B
:08F7C700784BE6F5993099FD3D
:10F7CF0090018B740AF090018BE0D39400748094B5
:09F7DF0080400600E014F080ED0A
:10F7E800C286800A7849E66406700375EF10784986
:0DF7F800E66407600302F0467880F6D2AFA9
:01F8050022E0
:103152007F0012346620090B7A007B327D017F00EA
:10316200122EDE300C0B7A007B1E7D017F00122EA8
:10317200DE300817300D147A007B327D01782CE6A0
:10318200FF122EDEC208122A37D209200B0C300D94
:1031920009788076F1122A37D20B300E0B300D08E7
:1031A200C20E1235C712F000200D121235D6E47B82
:0E31B2002C7A01F9F8C312100A5002D20D2235
:1034CF0075EF027F64EFD394007480948040031FE4
:1034DF0080F31217201235F612359FE4FFFE1234D7
:0934EF0027123152121A2E80F846
:10249E00005EBCE2613FDD83C29C7E20A3FD1F4136
:1024AE009DC3217FFCA2401E5F01E3BD3E6082DC26
:1024BE00237D9FC1421CFEA0E1BF5D0380DE3C6216
:1024CE00BEE0025CDF81633D7C22C09E1D43A1FF06
:1024DE004618FAA427799BC584DA3866E5BB5907F6
:1024EE00DB856739BAE406581947A5FB7826C49AE6
:1024FE00653BD987045AB8E6A7F91B45C6987A24D6
:10250E00F8A6441A99C7257B3A6486D85B05E7B9C5
:10251E008CD2306EEDB3510F4E10F2AC2F7193CDB5
:10252E00114FADF3702ECC92D38D6F31B2EC0E50A5
:10253E00AFF1134DCE90722C6D33D18F0C52B0EE95
:10254E00326C8ED0530DEFB1F0AE4C1291CF2D7385
:10255E00CA947628ABF517490856B4EA6937D58B75
:10256E005709EBB536688AD495CB2977F4AA481665
:10257E00E9B7550B88D6346A2B7597C94A14F6A855
:10258E00742AC896154BA9F7B6E80A54D7896B3545
:0A259E000000000000002B96B9DDDC
:03354000010F0A6E
:10359F0090018B1210BDFFFFFFFF90018BE0FCA38A
:0835AF00E0FDA3E0FEA3E0FF34
:0135B70022F1
:102BD70090FFFE121144ECF0A3EDF090FFFD1211EF
:0F2BE70044EBF0A3EAF0A3E9F090FFFC121144D5
:102BF600850883850982A3A3E4F085088385098275
:102C0600F0A3F0900007121168E0FEA3E0FF85082C
:102C160083850982E0FCA3E0FDC39FEE6480F8ECA7
:102C2600648098504C900004121168E0FBA3E0FA0F
:102C3600A3E0F98D828C83120ED6FF850883850961
:102C460082A3A3E06FFF900003121168EFF09000DB
:102C560003121168E090249E93850883850982A358
:102C6600A3F0850883850982E475F001120F6D8053
:0B2C760092850883850982A3A3E0FF7C
:062C81009000090211445D
:0E35B800CEEDCEEE6F7848F6E690249E93FF9F
:0135C60022E2
:1034F800EF7020F5A77598D0E589540F4420F58919
:10350800438E08CFEDCFEF90259D93F58DD28ED2C7
:05351800ACC2BCD2AF03
:01351D00228B
:1032DF0078121210A40000000078161210A400003B
:1032EF000000780A7664E47849F67849E6C39401D9
:1032FF0074809480502EE6FF25E025E0240BF8E43F
:10330F00F6EF25E025E0240CF8E4F6EF25E025E0C4
:10331F00240DF8E4F6EF25E025E0240EF8E4F67826
:04332F00490680C605
:013333002277
:10358300D2AFD2A9C2BBE589540F4401F589758E28
:0C35930002758CECE4F58AD28C0232DF69
:062B140090FFFF121144C6
:102B1A00850883850982E4F0850883850982E0FFB8
:102B2A00C39401748094804003022BD1EF25E025E1
:102B3A00E0240EF8E6FF7C00D39400748094804071
:102B4A0068E025E025E0240CF8E6705DEF30E00D42
:102B5A00D394017480948040047D0180087D0085AF
:102B6A000883850982E0FF123287850883850982F6
:102B7A00E0FF25E025E0240EF8E664017004FD126A
:102B8A003287850883850982E0FF25E025E0240E47
:102B9A00F816E66014EF25E025E0240DF8E6FEEFCE
:102BAA0025E025E0240CF8EEF6850883850982E005
:102BBA0025E025E0240CF8E66001168508838509DE
:072BCA0082E004F0022B225F
:062BD10090000102114416
:03000B00022F665B
:102F6600C0E0C0F0C083C082C0D0E8C0E0E9C0E0E5
:102F7600EAC0E0EBC0E0ECC0E0EDC0E0EEC0E0EFA0
:102F8600C0E0758CEC7812121080EF2401FFE43E4D
:102F9600FEE43DFDE43CFC781212108C780A16E63D
:102FA600701B7816121080EF2401FFE43EFEE43D0C
:102FB600FDE43CFC781612108C780A7664122B1409
:102FC60012351ED0E0FFD0E0FED0E0FDD0E0FCD010
:102FD600E0FBD0E0FAD0E0F9D0E0F8D0D0D082D053
:062FE60083D0F0D0E032C0
:10349B0090FFFF121144EDF090FFFF121144EFF07B
:1034AB00850883850982E0FFC39401748094805062
:1034BB000DA3E0FEEF25E025E0240BF8EEF69000DF
:0434CB0002021144A4
:102EDE0090FFFE121144EAF0A3EBF090FFFF1211E7
:102EEE0044EDF090FFFF121144EFF0850883850941
:102EFE0082E0FFC39401748094805056EF25E02544
:102F0E00E0240EF8E6704BE0FB25E025E0240CF8FB
:102F1E00E6703FA3E025E004FF850883850982E083
:102F2E00FA25E025E0240EF8EFF685088385098260
:102F3E00A3A3E0FEA3E0FF7C007D0A120F37EA2573
:102F4E00E025E0240DF8EFF6EB25E025E0240CF863
:082F5E00E4F6900004021144A6
:1032870090FFFF121144EDF090FFFF121144EFF091
:10329700850883850982E0FFFD7C00C39401748063
:1032A7009480501EEF25E025E0240BF8E66013A379
:1032B700E070047F0180027F00850883850982A36F
:1032C700EFF0ED4C700C850883850982A3E024FF9D
:0832D7009296900002021144DE
:0935D600C2AF7812121080D2AFCE
:0135DF0022C9
:0935E000C2AF7816121080D2AFC0
:0135E90022BF
:1034660090FFFF121144EFF0850883850982E07012
:10347600057810F608F6301216780FE675F064A493
:10348600FFC37811E69F18E695F05003E4F5D39054
:053496000001021144D9
:10356200D212E47810F608F6EF780F6003F68002C4
:10357200760AE4F5D975D2FF75D940F5D375EF0611
:013582002226
:0F35C700C212E47810F608F6780F76FFF5D922D5
:10351E00781106E618700106301216780FE675F06F
:10352E0064A4FFC37811E69F18E695F05003E4F506
:02353E00D32296
:0834270090018BEEF0A3EFF021
:10342F00E4A3F0A3F090018BE0FEA3E0FFC39001B3
:10343F008EE09F90018DE09E501C7FE87E03122F3F
:10344F00EC7F0112346690018EE004F070D790018A
:06345F008DE004F080CFB7
:013465002244
:082FEC009001A0EEF0A3EFF04C
:102FF400D394FAEE9400501D9001A0A3E0FFEFD308
:10300400940074809480405C000000000000000084
:1030140000001F80E99001A0E0FFA3E09001A3CF8E
:10302400F0A3EFF0D39001A4E094FA9001A3E0940C
:103034000040177FFA7E00122FEC9001A4E02406D2
:10304400F09001A3E034FFF080DAD39001A1E09482
:10305400009001A0E09400400B9001A3E0FEA3E0E7
:04306400FF122FEC3C
:013068002245
:102D300090019B7401F0A37401F0A37495F07B01E2
:062D40007A0179937D0287
:0E2D4600900197EBF0A3EAF0A3E9F0A3EDF003
:102D54007F0112346690019BE0FBA3E0FAA3E0F943
:102D6400120F832400FFE5F03460FE900197E0F930
:102D7400A3E0FAA3E090019EC9F0A3EAF0A3E9F06E
:102D8400E4FD90019AE0FCEDC39C5022EF2DF58206
:102D9400E43EF583E493FC90019EE0FBA3E0FAA3F8
:102DA400E0F98D82758300EC120F150D80D490012B
:102DB4009AE0FFA3E0FBA3E0FAA3E0F9E48FF002BA
:022DC4000FAE50
:10287A0090018D7412F0A37434F09001957401F0F4
:10288A00A37401F0A3748FF07B017A01798D7D0224
:0E289A00900191EBF0A3EAF0A3E9F0A3EDF0BA
:1028A8007880E664F160030229581235C7C2AFE4A4
:1028B800F5A7758F01A3E0FBA3E0FAA3E0F9120FD7
:1028C800832400FFE5F034607849F608EFF69001BC
:1028D80091E0FBA3E0FAA3E0F9784DC6EBC608C681
:1028E800EAC608C6E9C6E4784BF6900194E0FF789A
:1028F8004BE6C39F503C784DCBE6CB080806E6185C
:10290800CAE6CA70010614F9120EBD784CF675B7FE
:10291800A57880E6F5B7784CE6FF78490806E6180A
:10292800CCE6CC70010614F5828C83EFF0784B0668
:1029380080B8E4F58F900194E0FFA3E0FBA3E0FAF0
:10294800A3E0F9E48FF0120FAED2AFE4FF123562C4
:01295800225C
:103387007880E664F17048C2AF1235C7E4F5A775D7
:103397008F03784A766008F67849F67849E6C39449
:1033A7000874809480501F75B7A57880E6F5B778C4
:1033B7004AE6FE08E6F5828E83E4F026F6187402E4
:0F33C70036F6180680D5E4F58FD2AFFF123562C7
:0133D60022D4
:102A3700123387E490018FF0A3F07B019001950496
:102A4700F0A37401F0A3748FF01B7A00792E7D1622
:102A570012289A12287AE490018CF090018CE0C336
:102A6700781A964003022B0CE490018BF0900172C8
:102A7700E0FBA3E0FAA3E0F990018BE0FF75F0100B
:102A8700A4F58285F083120ED66071EF75F010A45D
:102A9700FF900172A3A3E02FF9EA35F0FA90000D39
:102AA7001210EE90018CE0FF782BE68FF0A429F945
:102AB700EA35F0FAEBC0E0EAC0E0E9C0E090017265
:102AC700E0FBA3E0FAA3E0F990018BE075F010A416
:102AD700F58285F083120ED6FD9001957401F0A35F
:102AE7007401F0A3748FF0D0E0F9D0E0FAD0E0FBE6
:102AF70012289A90018BE004F0022A7490018CE06E
:0C2B070004F0022A6212287AE47880F6BA
:012B1300229F
:0522420090018FEFF098
:10224700E4900195F0A3F0900192F07B0190019B3F
:1022570004F0A37401F0A37495F01B7A00792E7D26
:1022670016122D46122D30900193E0B4120CA3E004
:10227700B43407900192E04401F0E4900191F090AA
:102287000191E0C3781A964003022364E490019019
:10229700F0900172E0FBA3E0FAA3E0F9900190E06F
:1022A700FF75F010A4F58285F083120ED670030235
:1022B700235B90018FE0606AEF75F010A4FF900137
:1022C70072A3A3E02FF9EA35F0FA90000D1210EE91
:1022D700900191E0FF782BE68FF0A429F9EA35F019
:1022E700FAEBC0E0EAC0E0E9C0E0900172E0FBA3CE
:1022F700E0FAA3E0F9900190E075F010A4F582856B
:10230700F083120ED6FD90019B7401F0A37401F0C7
:10231700A37495F0D0E0F9D0E0FAD0E0FB122D4697
:102327008029900172E0FBA3E0FAA3E0F990019005
:10233700E075F010A4F58285F083120ED6FF9001A8
:1023470096E02FF0900195E03400F0900190E004C2
:10235700F0022298900191E004F0022286122D30BB
:10236700900193E0B4120CA3E0B43407900192E01B
:082377004402F0900192E0FF26
:01237F00223B
:1025A80048562B0048562D004856000418000001D4
:1025B800485600000000000001014904180000010D
:1025C80048564D656173000001014D01320000005D
:1025D800456E61626C6564000101510132000000C2
:1025E8004F6E30000000000001015201320000006F
:1025F8004F6E31000000000001015301320000005D
:102608004F6E32000000000001015401320000004A
:102618004F6E3300000000000101550406FA000166
:1026280049300000000000000101560406FA0001CC
:10263800493100000000000001015A0406FA0001B7
:10264800493200000000000001015E0406FA0001A2
:10265800493300000000000001016204180000096D
:1026680048564D6178000000010166041800000911
:10267800485653657400000001016A0406FA00090F
:10268800494F66730000000001016E000000000061
:0B269800000000000000000000000037
:10354300011A01430172FF25B34201400000440107
:0E35530045B0B8B1B941014200420143000049
:1030E300EF602A9001491210BD00000000900166B4
:1030F3001210BD4316000090016A1210BD000000BB
:10310300009001527401F0A3F0A3F0A3F0E4F5A73B
:1031130075A45D75A5FB75A60FD210FFFEFDFC120D
:10312300295990016A1210BD00000000C2A3C2A277
:10313300C2A1C2A0C29478347C007D007BFF30A67C
:0F314300067A2579A880047A2579AC12124122E8
:1027930090FFFF121144EFF0850883850982E070F2
:1027A30058FFFEFDFC900149E0F8A3E0F9A3E0FA2D
:1027B300A3E0FB120D85500A9001491210BD0000E1
:1027C3000000900166E0FCA3E0FDA3E0FEA3E0FFB0
:1027D300900149E0F8A3E0F9A3E0FAA3E0FB120DAE
:1027E3008560164014900166E0FCA3E0FDA3E0FEC3
:1027F300A3E0FF900149121098850883850982E0C0
:10280300FF7E0064037008900152E024FF92A3EF5F
:1028130064044E7008900153E024FF92A28508835C
:10282300850982E064057008900154E024FF92A1B9
:10283300850883850982E0FF7E00640670089001A5
:1028430055E024FF92A0EF640B4E7025FFFE7D162A
:102853007C43900166E0F8A3E0F9A3E0FAA3E0FB70
:10286300120D85600C400A9001661210BD431600DC
:072873000090000102114476
:08000300900185EFF07F00225F
:1033D700900185EBF0A3EAF0A3E9F0900185E0FB0B
:1033E700A3E0FAA3E0F9120EBDFF900188E0FBA36A
:1033F700E0FAA3E0F9EF120F03900185E0FBA3E0E9
:10340700FAA3E0F9900001120ED6FF900188E0FBC5
:10341700A3E0FAA3E0F9900001EF120F157F022253
:0823800090019BEEF0A3EFF0C9
:10238800C2837F017E00122FEC7F01123466E49035
:10239800019DF0A37408F090019DE0C39408748037
:1023A80094805038C280A3E05403940074809480D1
:1023B8004003D38001C392827F017E00122FECD2AA
:1023C800807F017E00122FEC90019EE0C313F07F06
:1023D8000112346690019DE004F080BB90019BE0FF
:1023E80090019FF0E490019DF0A37480F090019D0E
:1023F800E0C3940874809480503AC280A3E0FFA39D
:10240800E05F9400748094804003D38001C392827B
:102418007F017E00122FECD2807F017E00122FEC0C
:1024280090019EE0C313F07F0112346690019DE095
:1024380004F080B990019BA3E090019FF0E4900123
:102448009DF0A37480F090019DE0C394087480947B
:1024580080503AC280A3E0FFA3E05F9400748094A8
:10246800804003D38001C392827F017E00122FEC4B
:10247800D2807F017E00122FEC90019EE0C313F002
:102488007F0112346690019DE004F080B9D2837F09
:06249800017E00022FECA2
:0B1CB200900193EBF0A3EAF0A3E9F02F
:101CBD001235D6C8ECC8C9EDC9CAEECACBEFCB9068
:101CCD000141E02414FF900140E03400FEE4FCFDEE
:101CDD00C312100A50037F00221235D6900140EE38
:101CED00F0A3EFF0C280D282C2937F017E00122F4B
:101CFD00EC30810CD2937F017E00122FEC7F0022FD
:101D0D00E4900196F0A31210BD0000000090019622
:101D1D00E0C3942074809480504D7F017E00122F7B
:101D2D00ECD280900197E0FCA3E0FDA3E0FEA3E0E0
:101D3D00FF780112102FC8ECC8C9EDC9CAEECACB85
:101D4D00EFCBA281E4334BFFEAFEE9FDE8FC900105
:101D5D00971210987F017E00122FECC280C28290E4
:101D6D000196E004F080A6D280D282D293900197A2
:101D7D00E0FCA3E0FDA3E0FEA3E0FF781C12101B26
:101D8D00E47B03FAF9F8C3120FF4700D90019B1266
:101D9D0010BD3FA00000021E51900197E0FCA3E092
:101DAD00FDA3E0FEA3E0FF781C12101BEC4D4E4F7F
:101DBD00700BA31210BDBFA00000021E5190019721
:101DCD00E0FCA3E0FDA3E0FEA3E0FF781D12101BD5
:101DDD00E47B01FAF9F8C3120FF49001977010E04B
:101DED00FCA3E0FDA3E0FEA3E0FFEC540F800EE0AA
:101DFD00FCA3E0FDA3E0FEA3E0FFEC44F0FC9001AA
:101E0D0097121098900197E0FCA3E0FDA3E0FEA3CC
:101E1D00E0FFEC120DFE90019B121098E4FBFA7995
:101E2D0080784D90019BE0FCA3E0FDA3E0FEA3E0D4
:101E3D00FF120CE8E4FBFA79A0783F120BDF90015A
:101E4D009B12109830A639E4FFFE7DA07C3F9001D7
:101E5D009BE0F8A3E0F9A3E0FAA3E0FB120AEE90F1
:101E6D00019B12109890019BE0FCA3E0FDA3E0FE06
:101E7D00A3E0FF7B557A5579877842120BDF8055A9
:101E8D0090019BE0F8A3E0F9A3E0FAA3E0FBE4FFE7
:101E9D00FE7DA07C3F120AEA90019B1210989001E2
:101EAD009BE0FCA3E0FDA3E0FEA3E0FF7B557A558C
:101EBD0079877842120BDF90019B12109890019B4D
:101ECD00E0FCA3E0FDA3E0FEA3E0FFE4FBFA792034
:101EDD007840120AEA90019B12109890019BE0FC49
:101EED00A3E0FDA3E0FEA3E0FF900193E0FBA3E0E0
:091EFD00FAA3E0F91210427F0182
:011F060022B8
:0B132800900193EBF0A3EAF0A3E9F0C2
:101333001235D6C8ECC8C9EDC9CAEECACBEFCB90FB
:101343000144E02414FF900143E03400FEE4FCFD7B
:10135300C312100A50037F00221235D6900143EEC8
:10136300F0A3EFF0C280D282C2957F017E00122FDC
:10137300EC7F0112346630810CD2957F017E00121E
:101383002FEC7F0022900142E02401FFE433FE7C36
:10139300007D04120F3774452DF58274013CF583EB
:1013A300E0900197F05480D39400748094804003BC
:1013B300D38001C39282900197E0FF25E0F0E4908F
:1013C3000196F09001981210BD0000000090019664
:1013D300E0C394187480948050687F017E00122FBC
:1013E300ECD280900198E0FCA3E0FDA3E0FEA3E033
:1013F300FF780112102FC8ECC8C9EDC9CAEECACBD9
:10140300EFCBA281E4334BFFEAFEE9FDE8FC900158
:10141300981210987F017E00122FECC280900197E2
:10142300E0FF5480D39400748094804003D3800100
:10143300C39282EF25E0900197F0900196E004F0CB
:10144300808BD280D282D29520A60302154B9001C5
:1014530098E0FCA3E0FDA3E0FEA3E0FF78141210E4
:101463001BE47B03FAF9F8C3120FF4700280439074
:101473000198E0FCA3E0FDA3E0FEA3E0FF781412D3
:10148300101BEC4D4E4F700BA31210BD3FA000007C
:10149300021541900198E0FCA3E0FDA3E0FEA3E068
:1014A300FF781512101BE47B01FAF9F8C3120FF44D
:1014B300700D90019C1210BD0000000002154190B8
:1014C3000198A3E0FDA3E0FEA3E0FFED540FFDE4CC
:1014D300FC900198121098900198E0FCA3E0FDA302
:1014E300E0FEA3E0FF780412101B900198121098FD
:1014F300900198E0F8A3E0F9A3E0FAA3E0FBC3E4CA
:101503009BFFE49AFE740199FDE498FC9001981204
:101513001098900198E0FCA3E0FDA3E0FEA3E0FF98
:10152300EC120DFEE4FBFA79807847120CE8E4FB39
:10153300FA79A0783F120BDF90019C121098E4FB1C
:10154300FA797A7844021649900198E0FCA3E0FD09
:10155300A3E0FEA3E0FF781412101BE47B03FAF967
:10156300F8C3120FF4700D90019C1210BD3FD333DA
:1015730033021623900198E0FCA3E0FDA3E0FEA351
:10158300E0FF781412101BEC4D4E4F700BA312109A
:10159300BDBFD33333021623900198E0FCA3E0FDD3
:1015A300A3E0FEA3E0FF781512101BE47B01FAF918
:1015B300F8C3120FF49001987010A3E0FDA3E0FEAE
:1015C300A3E0FFED540FFDE4800FA3E0FDA3E0FED5
:1015D300A3E0FFED44F0FD74FFFC90019812109816
:1015E300900198E0FCA3E0FDA3E0FEA3E0FFEC1272
:1015F3000DFE90019C121098E4FBFA7980784990D3
:10160300019CE0FCA3E0FDA3E0FEA3E0FF120CE8D5
:10161300E4FBFA79A0783F120BDF90019C1210983B
:1016230090019CE0FCA3E0FDA3E0FEA3E0FFE4FB4C
:10163300FA79A0783F120AEE90019C1210987B0071
:101643007A40791C784690019CE0FCA3E0FDA3E07E
:10165300FEA3E0FF120CE87B007A24797478491228
:101663000BDF90019C12109890019CE0FCA3E0FD1D
:10167300A3E0FEA3E0FF90016EE0F8A3E0F9A3E08E
:10168300FAA3E0FB120AEA90019C121098E4FFFE11
:101693007DC87C4290019CE0F8A3E0F9A3E0FAA3A3
:1016A300E0FB120BDFE4FBFAF9783F120AEE122695
:1016B300A3E4FBFA79C87842120CE890019C12105B
:1016C3009890019CE0FCA3E0FDA3E0FEA3E0FFEC07
:1016D300C0E0EDC0E0EEC0E0EFC0E0900142E0FF0B
:1016E300C374039FFFE49400FE7802EFC333CE3349
:1016F300CED8F9FF900193E0FBA3E0FAA3E0F98FC2
:10170300828E83D0E0FFD0E0FED0E0FDD0E0FC127B
:0C171300105C900142E0045403F07F01E0
:01171F0022A7
:062959009001931210989A
:10295F0030A6257B557A5579877842900193E0FC14
:10296F00A3E0FDA3E0FEA3E0FF120CE8E4FBFA797D
:10297F00207840120CE88043E4FFFE7D207C4090DD
:10298F000193E0F8A3E0F9A3E0FAA3E0FB120AEE4B
:10299F007B557A5579877842120CE8E4FBFA792057
:1029AF007840120CE8C8ECC8C9EDC9CAEECACBEF23
:1029BF00CBE4FFFE7D807C3F120AEA900197121054
:1029CF0098E4FFFEFDFC900197E0F8A3E0F9A3E087
:1029DF00FAA3E0FB120D85500A9001971210BD006B
:1029EF00000000E4FFFE7D807C3F900197E0F8A39C
:1029FF00E0F9A3E0FAA3E0FB120D85600C400A900A
:102A0F0001971210BD3F8000007F007EFF7D7F7C0D
:102A1F0047900197E0F8A3E0F9A3E0FAA3E0FB12D7
:082A2F000BDF120E3C022380B4
:101A2E0030101A1235D6E47B2C7A01F9F8C3121055
:101A3E000A500AD2A3D2A2D2A1D2A0C2107B017A9E
:101A4E0001798B121CB2EF7003021C9A90018BE08D
:101A5E00FCA3E0FDA3E0FEA3E0FFEC30A62DC0E06A
:101A6E00EDC0E0EEC0E0EFC0E07B007A2479747840
:101A7E0049900156E0FCA3E0FDA3E0FEA3E0FF12B7
:101A8E000CE8E4FBFA797A7844802CC0E0EDC0E0F3
:101A9E00EEC0E0EFC0E07B007A24797478499001C3
:101AAE0056E0FCA3E0FDA3E0FEA3E0FF120CE87BF2
:101ABE00007A40791C7846120BDFC8ECC8C9EDC914
:101ACE00CAEECACBEFCBD0E0FFD0E0FED0E0FDD027
:101ADE00E0FC120AEA90018B121098E4FFFE7D7A68
:101AEE007C4490018BE0F8A3E0F9A3E0FAA3E0FBBD
:101AFE00120BDFE4FBFAF9783F120AEE1226A3E48A
:101B0E00FBFA797A7844120CE890018B121098E463
:101B1E00FFFEFDFC90018BE0F8A3E0F9A3E0FAA331
:101B2E00E0FB120D85500A90018B1210BD000000D3
:101B3E000090018BE0FCA3E0FDA3E0FEA3E0FF908C
:101B4E00014D121098E4FFFEFDFC900149E0F8A350
:101B5E00E0F9A3E0FAA3E0FB120D857017C2949092
:101B6E00016A1210BD000000007F007E007D007C27
:101B7E0000021C97E4FFFEFDFC900149E0F8A3E093
:101B8E00F9A3E0FAA3E0FB120D85500A9001491269
:101B9E0010BD00000000E4FFFE7D167C439001495D
:101BAE00E0F8A3E0F9A3E0FAA3E0FB120D85600CC8
:101BBE00400A9001491210BD43160000D2949001C4
:101BCE0049E0F8A3E0F9A3E0FAA3E0FBA3E0FCA34D
:101BDE00E0FDA3E0FEA3E0FF120AEA90018F1210CF
:101BEE009890016AE0FCA3E0FDA3E0FEA3E0FFEC09
:101BFE00C0E0EDC0E0EEC0E0EFC0E0E4FBFAF97843
:101C0E004090018FE0FCA3E0FDA3E0FEA3E0FF12F5
:101C1E000CE8C8ECC8C9EDC9CAEECACBEFCBD0E010
:101C2E00FFD0E0FED0E0FDD0E0FC120AEA90016A9F
:101C3E00121098E4FFFEFDFC90016AE0F8A3E0F9B3
:101C4E00A3E0FAA3E0FB120D85500A90016A121070
:101C5E00BD00000000E4FFFE7D1B7C4390016AE0A6
:101C6E00F8A3E0F9A3E0FAA3E0FB120D85600C40A7
:101C7E000A90016A1210BD431B000090016AE0FC3D
:101C8E00A3E0FDA3E0FEA3E0FF1229597B017A0138
:101C9E0079561213282087047F0180027F0090015D
:031CAE0051EFF003
:011CB1002210
:100AE700020EA8E86480F8E933E83360110460F087
:100AF700ED33EC337009E8FCE9FDEAFEEBFF220475
:100B070060DED3EB9FEA9EE99DE8C2E78CF0C2F76F
:100B170095F0400CE8CCF8E9CDF9EACEFAEBCFFB3B
:100B2700120E7385D0F05804700320D5B3E8047013
:100B3700075002B2D5020EB292D5EC0460F7E4CCAE
:100B4700C0E0C398F8603B94186008400DD0E0FB04
:100B5700020E8AE4FBFAC9FC8028E830E406E4C9FF
:100B6700FBE4CAFCE830E305E4C9CACBFCE8540758
:100B77006010F8C3E913F9EA13FAEB13FBEC13FC63
:100B8700D8F130F52FC3E49CFCEF9BFFEE9AFEED06
:100B970099FDD0E0FBEF4E4D4C701222DB03020EA5
:100BA700AFEC2CFCEF33FFEE33FEED33FDED30E71A
:100BB700EB020E8AEF2BFFEE3AFEED39FDD0E0FB9C
:100BC70050130BBB0003020EB2ED13FDEE13FEEF45
:080BD70013FFEC13FC020E8A6F
:100BDF00EC4D6011E8497017ED33EC3304600DE410
:100BEF00FCFFFEFD22E933E8330470F8020EA81271
:100BFF000E7358046009E4CC248150062850090272
:100C0F000EB2284003020EAFC0E0EB4A7044B98029
:100C1F0006D0E0FB020E9EEF4E701CBD8008EBFF6E
:100C2F00EAFEE9FD80EBE98DF0A4FEE5F0020CC8C9
:100C3F00E9CDF9EAFEEBFFEF89F0A4FCE5F0CE89F0
:100C4F00F0A42EFFE435F0CD89F0A42DFEE435F0AD
:100C5F008067EF4E7005BD80D780C3EF8BF0A4ACDB
:100C6F00F0EE8BF0A42CFCE435F0F8EF8AF0A42C16
:100C7F00E5F038FCE433CB8DF0A42CFCE5F03BF829
:100C8F00EE8AF0A42CFCE5F038F8E433CF89F0A419
:100C9F002CFCE5F038CF3400CE89F0A42FFFE5F01F
:100CAF003EFEE433C98DF0A42EFEE5F039CD8AF077
:100CBF00A42FFFE5F03EFEE43DFD33D0E0FB5007EF
:100CCF000BBB000F020EB2EC2CFCEF33FFEE33FE2A
:060CDF00ED33FD020E8A58
:100CE500020EB2EC5D046005E859047003020EA81B
:100CF500120E73580460F6EC4860F2EC7004FDFEC9
:100D0500FF22C860DB2481C85009C39860025006E1
:100D1500020EAF9850CAF582E9294B4A7005AB829D
:100D2500020E9E75F0007C1A7880C3EF9BEE9AED5B
:100D350099400DC3EF9BFFEE9AFEED99FDE842F059
:100D4500DC23ACF0D0E0FFD0E0FED0E0FDAB8220AC
:100D5500E7101BEB60BAEC2CFCEF33FFEE33FEED36
:100D650033FD020E8AE803F830E705C0F075F000A0
:100D7500EF2FFFEE33FEED33FD40B830E7C280AA1A
:100D850074F8CC6480CCC86480C8F58204604FC315
:100D9500EB9FF5F0EA9E42F0E99D42F0E89C45F0B4
:100DA500603C501DE5825FFFE582D313CB5BCBF43E
:100DB5002B5582FB50280ABA002409B90020088067
:100DC5001DE5825BFBE582D313CF5FCFF4C3132F01
:100DD5005582FF50090EBE00050DBD00010CC3EB89
:100DE5009FF5F0EA9E42F0E99D42F0E89C45F060EF
:090DF50007CC4820E701B3EC2211
:100DFE0075F020800E75F010800575F0087D007E70
:100E0E00007F003392D530D503120FE6EC3340103D
:100E1E00EF33FFEE33FEED33FDEC33FCD5F0ED2278
:0E0E2E00E5F0247EA2D513CC92E7CDCEFF22B4
:100E3C00EDD2E7CD33EC3392D524814006E4FFFEAE
:100E4C00FDFC22FCE4CFCECDCC24E0501174FF800D
:100E5C00EDC3CC13CCCD13CDCE13CECF13CF0470AA
:070E6C00F030D5DE020FE6B5
:1026A3009001A012109874FFFFFEFDFC9001A0E0C2
:1026B300F8A3E0F9A3E0FAA3E0FBC312100A603821
:1026C3007F807E967D187C4B9001A0E0F8A3E0F913
:1026D300A3E0FAA3E0FB120D856002501B7F807E0E
:1026E300967D187CCB9001A0E0F8A3E0F9A3E0FA73
:1026F300A3E0FB120D85500F9001A0E0FCA3E0FDC9
:10270300A3E0FEA3E0FF229001A0E0FCA3E0FDA371
:10271300E0FEA3E0FF120E3C9001A412109890017A
:10272300A4E0FCA3E0FDA3E0FEA3E0FFEC120DFE9A
:10273300C8ECC8C9EDC9CAEECACBEFCB9001A0E083
:10274300FCA3E0FDA3E0FEA3E0FF120AEAE4FBFA28
:10275300F9F8120D85602640249001A4E0FCA3E063
:10276300FDA3E0FEA3E0FFEF24FFFFEE34FFFEED49
:1027730034FFFDEC34FFFC9001A41210989001A4E7
:10278300E0FCA3E0FDA3E0FEA3E0FFEC120DFE22BC
:100E7300E9D2E7C933E833F892D5EDD2E7CD33ECC5
:070E830033FC5002B2D5223E
:100E8A00EC30E7100FBF000C0EBE00080DBD0004C9
:100E9A000BEB6014A2D5EB13FCED92E7FD2274FF75
:100EAA00FCFDFEFF22E480F8A2D574FF13FC7D80CE
:030EBA00E480EFE2
:03000000022E527B
:0C2E5200787FE4F6D8FD758181022E998E
:100EBD00BB010689828A83E0225002E722BBFE0233
:090ECD00E32289828A83E4932266
:100ED600BB010CE58229F582E5833AF583E02250D1
:100EE60006E92582F8E622BBFE06E92582F8E2221B
:0D0EF600E58229F582E5833AF583E4932235
:100F0300BB010689828A83F0225002F722BBFE01CD
:020F1300F322C7
:100F1500F8BB010DE58229F582E5833AF583E8F012
:100F2500225006E92582C8F622BBFE05E92582C8BE
:020F3500F222A6
:100F3700C2D5EC30E709B2D5E4C39DFDE49CFCEED5
:100F470030E715B2D5E4C39FFFE49EFE12128AC3B1
:100F5700E49DFDE49CFC800312128A30D507C3E4AC
:060F67009FFFE49EFE2244
:100F6D00C5F0F8A3E028F0C5F0F8E582158270020F
:060F7D001583E038F022AC
:100F8300BB010A89828A83E0F5F0A3E02250068739
:100F9300F009E71922BBFE07E3F5F009E3192289FB
:0B0FA300828A83E493F5F0740193222E
:100FAE00BB010789828A83020F6D500B09C5F0279A
:100FBE00F7C5F01937F722BBFE0D09F8E325F0F35C
:100FCE00C5F019E338F322F889828A8374019325D8
:080FDE00F0C5F0F8E49338229D
:0E0FE600C3E49FFFE49EFEE49DFDE49CFC221C
:100FF400EB9FF5F0EA9E42F0E99D42F0EC6480C874
:0610040064809845F02213
:10100A00EB9FF5F0EA9E42F0E99D42F0E89C45F03C
:01101A0022B3
:10101B00E86010ECA2E713FCED13FDEE13FEEF13EB
:04102B00FFD8F022D8
:10102F00E8600FEFC333FFEE33FEED33FDEC33FC1F
:03103F00D8F122C3
:10104200BB010789828A830210985005E9F80210D1
:0A1052008CBBFE05E9F80212F5223E
:10105C00BB010DE58229F582E5833AF583021098F0
:10106C005007E92582F802108CBBFE07E92582F8AF
:04107C000212F52245
:0C108000E6FC08E6FD08E6FE08E6FF229C
:0C108C00ECF608EDF608EEF608EFF62290
:0C109800ECF0A3EDF0A3EEF0A3EFF022CB
:1010A400D083D082E493F608740193F60874029313
:0910B400F608740393F67404734A
:1010BD00A8828583F0D083D0821210D41210D4125E
:1010CD0010D41210D4E473E493A3C583C5F0C58383
:1010DD00C8C582C8F0A3C583C5F0C583C8C582C87D
:0110ED0022E0
:1010EE00BB010DE58229F582E5833AF58302130AE9
:1010FE005007E92582F8021301BBFE07E92582F8A5
:10110E00021313E58229F582E5833AF58302131C57
:10111E00D083D082F8E4937012740193700DA3A360
:10112E0093F8740193F5828883E473740293686074
:06113E00EFA3A3A380DF74
:10114400E5092582F582E5083583F583B50804852C
:1011540082092210AF06858209F50822858209F5E5
:0411640008D2AF22DC
:0D116800E5092582F582E5083583F583222F
:10117500E709F60870FA8046E709F20870FA803E3A
:1011850088828C83E709F0A370FA807EE309F6086C
:1011950070FA8076E309F20870FA806E88828C8393
:1011A500E309F0A370FA806289828A83E0A3F608D6
:1011B50070FA805689828A83E0A3F20870FA804A21
:1011C50080D280FA80C680D4806580F2803180101C
:1011D50080A680EA809A80A880DA80E280CA803181
:1011E50089828A83ECFAE493A3C8C582C8CCC583F7
:1011F500CCF0A3C8C582C8CCC583CC70E9800D8965
:10120500828A83E493A3F60870F9ECFAA9F0EDFB62
:101215002289828A83ECFAE0A3C8C582C8CCC5833B
:10122500CCF0A3C8C582C8CCC583CC70EA80DD8963
:10123500828A83E493A3F20870F980CE88F0ED24C6
:1012450002B4040050C4F582EB2402B4040050BA81
:0912550023234582239011C57387
:1031C00090018FEBF0A3EAF0A3E9F0E4900197F00F
:1031D000A3F090019574FFF5F01212DF45F0603C0A
:1031E000900192E0FBA3E0FAA3E0F9120EBDFF907C
:1031F000018FE0FBA3E0FAA3E0F9900197E475F0FA
:10320000011212DF85F082F583EF120F15EF60C215
:10321000900193E475F001120F6D80B690018FE07C
:08322000FBA3E0FAA3E0F92290
:10306900900192EBF0A3EAF0A3E9F0A3EBF0A3EA55
:10307900F0A3E9F0900195E0FBA3E0FAA3E0F912CF
:103089000EBD600C900196E475F001120F6D80E49D
:10309900900195E0FBA3E0FAA3E0F9120EBD6D7073
:1030A9000122900192E0FBA3E0FAA3E0F9EBC0E072
:1030B900EAC0E0E9C0E0A3E0FBA374FFF5F0121257
:1030C900DFFAD082D083D0E06B7009E5F0658270B9
:0A30D90003EA658370BAFBFAF922DE
:10125E00EF4E6012EF60010EEDBB010B89828A83A7
:10126E00F0A3DFFCDEFA2289F05007F709DFFCA9B4
:0C127E00F022BBFEFCF309DFFCA9F0220B
:102E5E000234CFE493A3F8E493A34003F68001F287
:102E6E0008DFF48029E493A3F85407240CC8C33375
:102E7E00C4540F4420C8834004F456800146F6DF44
:102E8E00E4800B0102040810204080903540E47E5F
:102E9E00019360BCA3FF543F30E509541FFEE49339
:102EAE00A360010ECF54C025E060A840B8E493A300
:102EBE00FAE493A3F8E493A3C8C582C8CAC583CA2B
:102ECE00F0A3C8C582C8CAC583CADFE9DEE780BEE3
:013561000069
:10128A00BC000BBE0029EF8DF084FFADF022E4CC48
:10129A00F875F008EF2FFFEE33FEEC33FCEE9DEC11
:1012AA00984005FCEE9DFE0FD5F0E9E4CEFD22ED57
:1012BA00F8F5F0EE8420D21CFEADF075F008EF2FA1
:1012CA00FFED33FD4007985006D5F0F222C398FD92
:0512DA000FD5F0EA222F
:1012DF00A3F8E0C5F025F0F0E582158270021583C2
:0612EF00E0C838F0E8221F
:0C12F500ECF208EDF208EEF208EFF22235
:09130100E6FB08E6FA08E6F92211
:09130A00E0FBA3E0FAA3E0F922E4
:09131300E2FB08E2FA08E2F9220B
:0C131C00E493FB740193FA740293F9222D
:00000001FF
